:100000005228A301A200FF30A207031CA307031C70
:100010004D280330A100E6300F200328A101FC3E4B
:10002000A000A109031C1A28FF300000A007031834
:100030001528A0076400A10F14280800A2000630AC
:100040002128A80023082102031D282822082002B5
:10005000043003180130031902302805031DFF3056
:100060004D28A501A4011030A600210DA40DA50D59
:100070002208A4022308031C230FA5020318472803
:100080002208A40723080318230FA5070310A00DB7
:10009000A10DA60B352820084D28831303138312C6
:1000A0006400080083169B0183129F0183160730AA
:1000B0009C008601103085008312BA01BB013A080A
:1000C000B8003B08B9008A11842064008A11051E1B
:1000D0006B288A015F2864008A11051E6B28BA0A02
:1000E0000319BB0A3A08A0003B08A1002730A3006F
:1000F0000F308A011E208A11031D82280F30BA009A
:100100002730BB008A015F283808A0003908A10009
:10011000E830A2000330A3008A013120BC00380877
:10012000A0003908A100E830A2000330A3008A0132
:1001300031202408B8002508B9008A11F6203C08AF
:1001400086000830850001308A01012085013808C9
:10015000A0003908A1006430A200A3018A01312067
:10016000BC003808A0003908A1006430A200A30137
:100170008A0131202408B8002508B9008A11F62028
:100180003C0886000430850001308A010120850189
:100190003808A0003908A1000A30A200A3018A0192
:1001A0003120BC003808A0003908A1000A30A200A4
:1001B000A3018A0131202408B8002508B9008A115A
:1001C000F6203C0886000130850001308A010120BC
:1001D00085013808BC008A11F6203C0886000230F0
:1001E000850001308A010120850108003C08093C96
:1001F0008A11031C0E298A110021BC008A110E29C4
:1002000001308A003C08820722347B3416341A34C9
:100210004B348A34C2343B3402340B34080063005C
:040220008A010F2917
:02400E00423F2F
:00000001FF
